:100000000C9468000C944F0D0C94780D0C948500A2
:100010000C9485000C9485000C94C40C0C94A00CDA
:100020000C94A20A0C9485000C9485000C9468072B
:100030000C9499070C9485000C94140F0C94850073
:100040000C9485000C9485000C9485000C9485001C
:100050000C948500DB0F2710380F27102710420F54
:100060004C0F2710510F271027105B0F650F27101B
:100070006A0F27102710740F7E0F2710830F271089
:1000800027108C0F950F27109A0F27102710A40FF9
:10009000AE0F2710B30F27102710BD0FEA0F271040
:1000A000C70F27102710D10FDB0F2710E00F2710E5
:1000B0002710E50FEA0F2710EF0F27102710F90F71
:1000C00003102710051013101610271027101910F1
:1000D00011241FBECFE5D4E0DEBFCDBF10E0A0E607
:1000E000B0E0EAE2FCE202C005900D92A636B1074C
:1000F000D9F711E0A6E6B0E001C01D92A633B10722
:10010000E1F70E94FB030C9413160C9400001F935C
:10011000182F682F617081E00E94A50D612F627019
:1001200082E00E94A50D612F647083E00E94A50DFE
:1001300084E060E00E94A50D1F910895CF93DF93A6
:1001400060B3647082E00E94A50D60B3687083E0C4
:100150000E94A50D60B370E07695679576956795DA
:10016000C1E0D0E06C277D27617081E00E94A50D81
:1001700060B370E083E0769567958A95E1F76C2728
:100180007D27617084E00E94A50D0E94950E882352
:1001900009F44BC00E94EF0A882309F446C0813459
:1001A00031F480916A00823084F48F5F0CC0823415
:1001B00019F410926A0009C0833439F480916A00FE
:1001C0008F3F1CF0815080936A0080916A008E3FBF
:1001D00039F488E19CEF0E94120C88E19CEF23C067
:1001E0008F3F39F48CE09EEF0E94120C8CE09EEF62
:1001F0001AC0882339F480E090E00E94120C80E05D
:1002000090E011C0813039F484EF91E00E94120C2B
:1002100084EF91E008C0823041F488EE93E00E94C0
:10022000120C88EE93E00E94590CDF91CF91089553
:100230000E94EC0A882319F00E94870067C0809111
:100240006000909161009C012F5F3F4F30936100EF
:100250002093600023E08032920709F44AC023E033
:1002600081329207C0F421E0843F9207D9F121E066
:10027000853F920730F421E08039920709F04CC0A5
:1002800024C022E08835920779F122E08C3B920766
:1002900009F042C02BC024E08C34920781F124E0A5
:1002A0008D34920748F423E08438920721F123E04B
:1002B000883E920789F521C024E0803B920709F12E
:1002C00025E08431920741F521C081E060E00E9481
:1002D000A50D82E060E00E94A50D83E060E00E9431
:1002E000A50D0FC081E003C081E00CC082E061E099
:1002F0000AC082E007C083E0FACF83E003C084E055
:10030000F6CF84E060E00E94A50D06C080E991E090
:1003100090936100809360008AE090E00E94441511
:100320000895CF92DF92EF92FF920F931F93CF9396
:10033000DF930E94EC0A882309F456C0803829F420
:1003400053C08AE090E00E9444150E94EC0A882382
:10035000C1F760E080916600882309F461E0609352
:10036000660080E00E94A30E60E08091660081112B
:1003700061E081E00E94A30E60E08091660081113F
:1003800061E082E00E94A30E60E08091660081112E
:1003900061E087E00E94A30E60E080916600882300
:1003A00009F461E083E00E94A30E60E080916600A2
:1003B000882309F461E084E00E94A30E60E080914C
:1003C0006600882309F461E085E00E94A30E60E0E6
:1003D00080916600882309F461E086E00E94A30E04
:1003E00084E690E00E94441580916600882349F1DC
:1003F00080E062E00E94470E7C0182E062E00E94A1
:10040000470EEC0181E062E00E94470E10E08A3165
:10041000910508F011E060E08AE1E816F10408F0C7
:1004200061E081E00E94A50D82E0612F0E94A50D90
:1004300083E0612F0E94A50D60E0CA31D105A0F1D3
:1004400032C083E062E00E94470E8C0184E062E0EB
:100450000E94470EEC0185E062E00E94470E7C019D
:1004600086E062E00E94470E6C0160E08AE1E816D7
:10047000F10408F061E081E00E94A50D60E00A311E
:10048000110508F061E082E00E94A50D60E0CA312C
:10049000D10508F061E083E00E94A50D60E08AE1EB
:1004A000C816D10408F061E084E00E94A50DDF9138
:1004B000CF911F910F91FF90EF90DF90CF90089513
:1004C0000E94C50B0E94E70B08951F93982F9295E9
:1004D0009F70182F1F709A301CF4892F805D02C006
:1004E000892F895A1A3014F4105D01C0195A0E94DC
:1004F000F006812F0E94F0061F91089588B3817E37
:1005000088BB82E390E00E94441588B3817E88BB5B
:1005100082E390E00E94441508950F931F93082FE3
:1005200014E010C0802F61E00E94A50D80E590E0EE
:100530000E944415802F60E00E94A50D88E790E09E
:100540000E944415115070F71F910F9108951F9349
:1005500083E00E948D0210E0812F61E00E94A30ED3
:100560001F5F1830C9F783E0809366001F910895DC
:1005700083E061E00E94A30E84E061E00E94A30E8C
:1005800085E061E00E94A30E86E061E00E94A30E78
:1005900081E00E948D02089582E00E948D020895FC
:1005A0000F931F93082F1AE010C0802F61E00E9464
:1005B000A50D88E290E00E944415802F60E00E9423
:1005C000A50D8CE390E00E944415115070F71F9127
:1005D0000F9108952F923F924F925F926F927F9268
:1005E0008F929F92AF92BF92CF92DF92EF92FF9243
:1005F0000F931F93DF93CF9300D00F92CDB7DEB749
:100600000E948E0E0E94EC0A882369F480916B0090
:1006100010926B00813081F0823009F4CAC08430BE
:1006200009F0C5C0C1C0803809F4C1C090916B0009
:10063000982B90936B00BBC00E947E020E942805FD
:100640000E94AD0681E00E94D00241E049830E94F1
:1006500039061B01C82E0E940206162FF72EE82E1F
:10066000D92E20E030E040E050E004E10E94E513A4
:100670009B838A83612F7F2D8E2D9D2D2FEF30E060
:1006800040E050E00E94E5135C01612F7F2D8E2D2C
:100690009D2D27EB34EF4AEB50E00E94E5134C010F
:1006A000612F7F2D8E2D9D2D28E535EB41E950E002
:1006B0000E94E5133C01612F7F2D8E2D9D2D2AEA8E
:1006C0003FEC47E250E00E94E5132C01612F7F2DA3
:1006D0008E2D9D2D2CEF3BEE4CE050E00E94E5135B
:1006E0009501EA81FB81EA15FB0508F49F0182165A
:1006F000930608F494016216730608F493014216F7
:10070000530608F492018217930708F49C01F3E062
:1007100024383F0700F54A815B812417350711F41F
:1007200081E01AC02A153B0511F482E015C0281596
:10073000390511F489E010C02615370511F486E05B
:100740000BC02415350511F483E006C028173907BE
:1007500011F48CE001C080E098B3880F917E892B62
:1007600088BB5981533089F580E20E94F00683E20C
:100770000E94F0068C2D0E946502832D0E94650266
:10078000822D0E94650284E20E94F0068E2D0E9456
:1007900065028F2D0E946502812F0E94650284E60A
:1007A00090E00E94441511C083E0898350CF1982E4
:1007B0004ECF0E947E020E94C3040E94AD0682E0DA
:1007C0000E94D002E2E0E98342CF0F900F900F9099
:1007D000CF91DF911F910F91FF90EF90DF90CF901D
:1007E000BF90AF909F908F907F906F905F904F9051
:1007F0003F902F9008951F9387B38E6187BB80E051
:1008000096E90E94BF060E9463070E94F00B0E94B7
:10081000940A0E94E80C0E945F10789484E690E0AD
:100820000E94441586E50E94F00680E30E94F006CF
:1008300082E30E94F00680E20E94F00680E20E94BD
:10084000F00680E20E94F0060E94B60610E0812FBA
:1008500060E00E94A30E1F5F1830C9F784E690E0A5
:100860000E9444150E94EC0A182F882321F41EC010
:10087000812F0E9487000E94EC0A8823C9F70E94FA
:100880008700113029F40E94B8020E949101FDCF27
:10089000123029F40E94CC020E949E00FDCF143039
:1008A00029F40E94A7020E94EA02FDCF0E94600282
:1008B0000E941801FDCFEF92FF920F931F93CF93E9
:1008C000DF93E82FF0E021E930E0EF01CC0FDD1FEE
:1008D000D901AC0FBD1F0D911C9111974CE6E42E70
:1008E00040E0F42EEC0EFD1E3596EE0FFF1FE20FDA
:1008F000F31F20813181201B310B40E050E060E08C
:1009000070E080E890E00E949415F7013183208325
:10091000CA58DF4F85E0169507958A95E1F7198348
:100920000883DF91CF911F910F91FF90EF90089571
:1009300080E00E945B0481E00E945B0482E00E94F0
:100940005B0483E00E945B0484E00E945B040895E2
:10095000EF92FF921F93CF93DF93182F61E00E94D5
:10096000470EEC01812F60E00E94470EC81BD90B97
:10097000D7FF02C0C0E0D0E0CE01DF91CF911F9140
:10098000FF90EF9008951F93CF93DF9310929C00F8
:1009900010929B0010929E0010929D001092A00059
:1009A00010929F001092A2001092A1001092A40039
:1009B0001092A30010E00E948E0EC0919B00D09177
:1009C0009C0080E00E94A804C80FD91FD0939C000F
:1009D000C0939B00C0919D00D0919E0081E00E9439
:1009E000A804C80FD91FD0939E00C0939D00C0914A
:1009F0009F00D091A00082E00E94A804C80FD91FD8
:100A0000D093A000C0939F00C091A100D091A200FC
:100A100087E00E94A804C80FD91FD093A200C093FA
:100A2000A100C091A300D091A40088E00E94A80476
:100A3000C80FD91FD093A400C093A3001F5F10322A
:100A400009F0B9CF0E949804DF91CF911F910895CA
:100A50001F93CF93DF931092920010929100109207
:100A600094001092930010929600109295001092AC
:100A700098001092970010929A001092990010E03E
:100A80000E948E0EC0919100D091920080E00E9451
:100A9000A804C80FD91FD0939200C0939100C091B1
:100AA0009300D091940081E00E94A804C80FD91F40
:100AB000D0939400C0939300C0919500D09196007C
:100AC00082E00E94A804C80FD91FD0939600C0935B
:100AD0009500C0919700D091980087E00E94A804EB
:100AE000C80FD91FD0939800C0939700C091990068
:100AF000D0919A0088E00E94A804C80FD91FD09313
:100B00009A00C09399001F5F103209F0B9CF0E947C
:100B10009804DF91CF911F9108951F93182F833070
:100B200038F0873029F0883019F060E070E031C08B
:100B3000812F0E94A804133008F01450E12FF0E038
:100B4000DF01AA0FBB1FAA58BF4F2D913C911197EF
:100B50008217930708F49C01821B930BBC0180E071
:100B600090E0EE0FFF1FE459FF4F2081318140E0FC
:100B700050E00E944E15672F782F892F99276030FB
:100B800020E8720720E0820720E0920710F06FEF64
:100B90007FE7CB011F9108951F93182F833038F002
:100BA000873029F0883019F060E070E028C0812F8C
:100BB0000E943B0E133008F01450282F392F37FFB6
:100BC00002C020E030E040E050E0E12FF0E0EE0F26
:100BD000FF1FE459FF4F6081718180E090E00E9427
:100BE0004E15672F782F892F9927603020E87207DC
:100BF00020E0820720E0920710F06FEF7FE7CB0143
:100C00001F9108950F931F93CF93DF9382E00E946B
:100C10008D058C0181E00E948D05EC0180E00E9431
:100C20008D0516950795169507950F3F110519F037
:100C300010F00FEF10E0BE017695679576956795F9
:100C40006F3F710519F010F06FEF70E0AC01569531
:100C50004795569547954F3F510519F010F04FEFC6
:100C600050E0802F0E947F14DF91CF911F910F9150
:100C700008950F931F93CF93DF9382E00E948D0519
:100C80008C0181E00E948D05EC0180E00E948D05C1
:100C900016950795169507950F3F110519F010F059
:100CA0000FEF10E0BE0176956795769567956F3FDB
:100CB000710519F010F06FEF70E0AC015695479593
:100CC000569547954F3F510519F010F04FEF50E002
:100CD000802F0E941F15DF91CF911F910F910895D2
:100CE00064E171E081E092E041E950E00E94471345
:100CF000882381F580E090E490939C0080939B0092
:100D000020E030E630939E0020939D009093A00059
:100D100080939F0080E09AE09093A2008093A100CE
:100D20009093A4008093A30080E890E090939200B9
:100D300080939100909394008093930090939600F9
:100D400080939500909398008093970090939A00D9
:100D5000809399000E949804089564E171E081E015
:100D600092E041E950E00E94E01208958091220152
:100D700080FD02C00E945F100E94700608959C01D1
:100D800040E050E084E0220F331F441F551F8A9536
:100D9000D1F760EC71EE84EE90E00E949415215042
:100DA000304030BD29B90895F894E091A700F0E0F3
:100DB000E854FF4F80819091A600983021F49091E3
:100DC000A7009093A6009091A7009F5F9093A70023
:100DD0009091A700983010F01092A7007894089591
:100DE000F894E091C000F0E0E855FF4F80839091C7
:100DF000C0009F5F9093C0009091C000903110F0B0
:100E00001092C0002091C0009091A500291719F4FC
:100E100090E19093C000559A78940895CF93DF9312
:100E2000EC0107C09091C0009031E1F321960E943F
:100E3000F00688818823B1F7DF91CF910895CF9391
:100E4000DF93EC0106C09091C0009031E1F30E9465
:100E5000F006FE01219684918823A9F7DF91CF91B6
:100E600008950F931F93CF93DF93EC018B0109C07B
:100E70008091C0008031E1F389910E94F006015019
:100E8000104001151105A1F7DF91CF911F910F912E
:100E900008950F931F93CF93DF93EC018B010BC049
:100EA0008091C0008031E1F3FE01219684910E947F
:100EB000F006015010400115110591F7DF91CF9117
:100EC0001F910F91089588EB8AB908951AB8089573
:100ED0001F920F920FB60F9211248F939F93EF934F
:100EE000FF938CB19091A6009830D1F0E091A600CC
:100EF000F0E0E854FF4F80838091A6008F5F8093DD
:100F0000A6008091A600883010F01092A600909163
:100F1000A6008091A700981719F488E08093A60096
:100F2000FF91EF919F918F910F900FBE0F901F90A7
:100F300018951F920F920FB60F9211248F939F93C3
:100F4000EF93FF939091A5008091C0009817D9F07E
:100F5000E091A500F0E0E855FF4F90818091C0003E
:100F6000803121F48091A5008093C0008091A5007C
:100F70008F5F8093A5008091A500803110F01092C2
:100F8000A5009CB901C05598FF91EF919F918F9159
:100F90000F900FBE0F901F90189510928300109223
:100FA00082001092850010928400109287001092A7
:100FB0008600109289001092880010928B00109287
:100FC0008A0010928D0010928C00089524E0880F02
:100FD000991F2A95E1F7909387008093860084E01B
:100FE000660F771F8A95E1F770938D0060938C00F0
:100FF0000895DF93CF930F92CDB7DEB79091CE00D7
:10100000981731F089830E94CD0789818093CE00A3
:101010000F90CF91DF9108958091C700882371F1DF
:101020008091EC009091ED002091EA003091EB006E
:10103000821B930B2091C3003091C400821B930B41
:101040008B30910514F08AE090E02FEF863F9207F5
:1010500014F486EF9FEF282F220F220F280F2093E2
:10106000C8001816190614F481E005C0009711F4A1
:1010700080E001C08FEF8093D50008951092D500D5
:101080001092C800089580E00E94F90708950F9318
:101090001F93CF93DF93EC018B0183E00E94F9074C
:1010A000D093D100C093D0001093C6000093C50028
:1010B000DF91CF911F910F910895EF92FF920F93BF
:1010C0001F93CF93DF93EC018B017A0184E00E94A0
:1010D000F907F0926300E09262008091EA0090913B
:1010E000EB008C0F9D1F9093D1008093D0008091D6
:1010F000EC009091ED00800F911F9093C6008093BB
:10110000C5001092C700C017D10719F481E0809381
:10111000C7008091EC009091ED002091EA003091A1
:10112000EB00821B930B9093C4008093C300DF916C
:10113000CF911F910F91FF90EF9008952091EA00B9
:101140003091EB00E091EC00F091ED006E1B7F0B15
:10115000821B930B0E945D080895EF92FF920F93FC
:101160001F93CF93DF938091CE0082FD03C000E0F8
:1011700010E020C00091D0001091D10080E00E94CA
:101180001D0DEC01E090C500F090C60080E00E94CB
:10119000360DE81AF90AF7FE04C0F094E194F1085C
:1011A000F3940C1B1D0B17FF03C0109501951F4FE7
:1011B0000E0D1F1DC801DF91CF911F910F91FF9060
:1011C000EF900895CF93DF939091EE0082E3980221
:1011D000C00111244091C9005091CA009A01220F08
:1011E000331F240F351F820F931F64E070E00E94AD
:1011F00081159B017093CA006093C9004091C100A2
:101200005091C200CA01880F991F840F951F820F49
:10121000931F64E070E00E9481157093C200609398
:10122000C1004091CE00442309F495C08091C500CF
:101230009091C600443051F56091EC007091ED0042
:101240004091620050916300861B970B4817590725
:101250000CF4CA0166277727641B750B861797075E
:101260000CF4CB014091D500552747FD5095841BC8
:10127000950B61F410928D0010928C0010928B00EF
:1012800010928A001092890010928800A091880024
:10129000B091890040918A0050918B0060918C0040
:1012A00070918D00E0E460307E071CF060E070E437
:1012B00006C0E0EC61307E0714F460E070ECF901E8
:1012C000EE0FFF1FEA01CE1BDF0BFE01E80FF91F37
:1012D000CF01880F991FEE0FFF1FEE0FFF1FEE0FBC
:1012E000FF1F8E0F9F1F440F551F4A1B5B0B421B96
:1012F000530BFA01A3E0EE0FFF1FAA95E1F7E41BE1
:10130000F50B8E0F9F1F860F971F90938D00809374
:101310008C0040918A0050918B005093890040933B
:10132000880030938B0020938A0060E170E00E9477
:101330008115CB012091C800332727FD3095821BF2
:10134000930B1816190614F4889603C0009709F039
:1013500088970E94590C1092EE00DF91CF9108956A
:10136000882361F080E00E94F90780E090E00E940D
:10137000590C80E090E00E94120C089580E090E00B
:1013800060E070E00E9447080895CF93DF9390914A
:10139000E70082E39802C00111244091D2005091ED
:1013A000D3009A01220F331F240F351F820F931F82
:1013B00064E070E00E9481159B017093D3006093FC
:1013C000D2004091CC005091CD00CA01880F991FE6
:1013D000840F951F820F931F64E070E00E948115B7
:1013E0007093CD006093CC004091CE00442309F46B
:1013F00096C08091D0009091D100443061F5409129
:10140000EA005091EB006091620070916300841BD0
:10141000950B681779070CF4CB01EE27FF27E61B25
:10142000F70BAC018E179F070CF4AF018091D5002C
:10143000992787FD9095840F951F009761F410926E
:1014400087001092860010928500109284001092FE
:10145000830010928200A0918200B091830040919D
:101460008400509185006091860070918700E0E4CF
:1014700060307E071CF060E070E406C0E0EC613094
:101480007E0714F460E070ECF901EE0FFF1FEA0133
:10149000CE1BDF0BFE01E80FF91FCF01880F991F4C
:1014A000EE0FFF1FEE0FFF1FEE0FFF1F8E0F9F1F90
:1014B000440F551F4A1B5B0B421B530BFA01A3E061
:1014C000EE0FFF1FAA95E1F7E41BF50B8E0F9F1F90
:1014D000860F971F90938700809386004091840029
:1014E0005091850050938300409382003093850093
:1014F0002093840060E170E00E9481158091C80013
:10150000992787FD9095860F971F1816190614F4D2
:10151000889603C0009709F088970E94120C1092D9
:10152000E700DF91CF9108958091220181FD02C0F3
:101530000E94F00B89B7846089BF0E94CD0710928A
:10154000CE0008951F920F920FB60F9211242F9381
:101550003F934F935F936F937F938F939F93AF933B
:10156000BF93EF93FF9380918100982F9F5F90939B
:101570008100209180002223F1F421E0209380005B
:101580009F3040F08E508093810081E066E170E0F2
:101590000E9474118091CF008F5F8093CF008339B8
:1015A00040F00E940C080E94C5090E94E2081092B7
:1015B000CF0010928000FF91EF91BF91AF919F916A
:1015C0008F917F916F915F914F913F912F910F90EC
:1015D0000FBE0F901F9018958091D600089520910E
:1015E000DF00922F992311F493E001C09150E92F6D
:1015F000F0E0E552FF4F8081882311F010820895BA
:10160000921781F708954FB7F89420910601309111
:10161000070180911C0190911D014FBF42E02D3DBB
:101620003407B8F5821B930B97FF03C09095819503
:101630009F4F8430910568F5369527953695279507
:101640006091DA00269FA00111245093E1005C35DF
:1016500058F0513818F05F39E0F42CC0503710F4CE
:1016600086E01DC082E01BC0573430F05C3410F4BB
:1016700085E015C081E013C0513410F083E00FC045
:101680005C3328F480E893E09093E00010C087E09A
:1016900006C083E08093E0001092D60008959091F8
:1016A000E000992321F091509093E00080E880932E
:1016B000D600089584E0F3CF8091D600803809F4F5
:1016C00046C09091D900982709F441C090FF13C0FB
:1016D00080FD02C031E601C031E42091DF00E22F3D
:1016E000F0E0E552FF4F30832F5F2093DF0024307E
:1016F00010F01092DF0091FF13C081FD02C032E6AE
:1017000001C032E42091DF00E22FF0E0E552FF4F0C
:1017100030832F5F2093DF00243010F01092DF0021
:1017200092FF13C082FD02C023E601C023E4909122
:10173000DF00E92FF0E0E552FF4F20839F5F909399
:10174000DF00943010F01092DF008093D9000895EC
:101750006091D7007091D80082E06C3D780718F452
:101760006CED72E006C083E0603D780710F06FEC2E
:1017700073E0769567957695679580E89BEB70E0CA
:101780000E946D156093DA0008958CE792E9019745
:10179000F1F780910601909107019093D800809312
:1017A000D7000E94A80B089562E071E081E092E00A
:1017B00047ED50E00E944713882331F48CED92E00E
:1017C0009093D8008093D7000E94A80B089562E000
:1017D00071E081E092E047ED50E00E94E012089550
:1017E0008091220182608093220182B3806F82BB4C
:1017F00081B3806F81BB82EF8FBD81E08EBD89B7E1
:1018000089BF08958FB7F8941092E4001092E30016
:101810001092E6001092E5001BBC1ABC19BC18BC63
:101820008FBF089562E070E00E948115862F972F88
:1018300022E0803092071CF08FEF91E006C02EEF7F
:10184000813092077CF097FD0FC09093E400809365
:10185000E300969B04C08091E200827015C099BDA0
:1018600088BD089581E09EEF22273327281B390B7E
:101870003093E4002093E300969B03C039BD28BD5C
:1018800008958091E20081608093E20019BC18BC49
:1018900089B7886089BF08952091E3003091E40002
:1018A000220F331F969B03C0309521953F4FC901EE
:1018B000089562E070E00E948115862F972F22E044
:1018C000803092071CF08FEF91E006C02EEF813040
:1018D00092077CF097FD0FC09093E6008093E5009F
:1018E000979B03C09BBD8ABD08958091E2008260F2
:1018F0000FC081E09EEF22273327281B390B30933E
:10190000E6002093E500979B0BC08091E200817078
:101910008093E2001BBC1ABC89B7806189BF08951F
:101920003BBD2ABD08952091E5003091E600220FCD
:10193000331F979903C0309521953F4FC9010895F2
:101940001F920F920FB60F9211248F939F93849B37
:1019500014C082B39091E20090FD02C090E001C0FB
:1019600090E48F7B892B82BB8091E3009091E4000F
:1019700099BD88BD89B7877F89BF9F918F910F904F
:101980000FBE0F901F9018951F920F920FB60F92D7
:1019900011248F939F93859B14C082B39091E20092
:1019A00091FD02C090E001C090E88F77892B82BB47
:1019B0008091E5009091E6009BBD8ABD89B78F7E3E
:1019C00089BF9F918F910F900FBE0F901F90189518
:1019D00085B78F6085BF8BB7806C8BBF9698979AC1
:1019E00008958FB7F8942091EA003091EB0030937E
:1019F000F0002093EF002091EC003091ED00309347
:101A0000E9002093E8008FBF08958FB7F8942091E4
:101A1000EA003091EB003093F0002093EF008FBF8D
:101A200008958FB7F8942091EC003091ED00309339
:101A3000E9002093E8008FBF08959FB7F8942091A4
:101A4000EA003091EB004091EF005091F0008823C4
:101A500041F06091EA007091EB007093F0006093A8
:101A6000EF009FBF241B350BC90108959FB7F89461
:101A70002091EC003091ED004091E8005091E90098
:101A8000882341F06091EC007091ED007093E900C3
:101A90006093E8009FBF241B350BC90108951F9276
:101AA0000F920FB60F9211248F939F93969B0BC0AA
:101AB0008091E70081508093E7008091EA00909147
:101AC000EB0001970AC08091E7008F5F8093E700E9
:101AD0008091EA009091EB0001969093EB00809347
:101AE000EA009F918F910F900FBE0F901F90189555
:101AF0001F920F920FB60F9211248F939F93979B73
:101B00000BC08091EE008F5F8093EE008091EC001F
:101B10009091ED0001960AC08091EE008150809373
:101B2000EE008091EC009091ED0001979093ED0014
:101B30008093EC009F918F910F900FBE0F901F909C
:101B4000189587B38E6187BB08956623A1F0823014
:101B500061F0833018F4813009F505C0833039F025
:101B60008430E1F406C0C19A0895C29A0895C39AD8
:101B70000895C49A0895823061F0833018F481305A
:101B800069F405C0833039F0843041F406C0C1984F
:101B90000895C2980895C3980895C498089582300E
:101BA00069F0833018F48130A9F405C0833049F01E
:101BB000843081F40BC088B392E005C088B394E010
:101BC00002C088B398E0892788BB089588B390E164
:101BD000892788BB0895823081F0833018F48130E2
:101BE00029F406C0833081F08430B9F080E0089594
:101BF00088B390E0969587950EC088B390E096954F
:101C000087959695879507C088B390E033E09695C1
:101C100087953A95E1F78170089588B390E024E0C4
:101C2000969587952A95E1F781700895882311F498
:101C300070E001C072E0662311F450E001C054E08E
:101C4000442311F430E001C038E0222311F490E085
:101C500001C090E12FB7F89488B3817E872B852B44
:101C6000832B892B88BB2FBF08953398379808950D
:101C7000379A339A08959FB7F8949FBFE82FF0E002
:101C8000EE0FFF1FEC50FF4F808191810895662376
:101C900061F49FB7F894E82FF0E0EE0FFF1FEC50CF
:101CA000FF4F208131819FBF2FC0613081F49FB7EA
:101CB000F894855FE82FF0E0EE0FFF1FEC50FF4F28
:101CC000308121819FBFC901292F382F1DC062306B
:101CD000C9F49FB7F8949FBFA82FA55FB0E0AA0FE3
:101CE000BB1FAC50BF4FE82FF0E0EE0FFF1FEC50D2
:101CF000FF4F2D913C91119780819181281B390BC9
:101D000037FF02C020E030E0C90108958FB7F89492
:101D10008FBF809120019091210108958091F3005F
:101D20009091F3008917E1F308958091F300909169
:101D30008E00981711F480E008958091F30080934D
:101D40008E0081E00895883011F487E003C0893067
:101D500008F066C02091F200662351F141E050E0A6
:101D6000082E02C0440F551F0A94E2F7242B20933B
:101D7000F2008430A9F0853038F4823079F0833075
:101D8000A8F4813039F408C0863071F0863050F004
:101D9000873061F0DA9832C0DD9824C0D89824C02A
:101DA000D99824C0DF9824C0DB9824C0DE9824C0D2
:101DB000422F50E0082E02C0559547950A94E2F74D
:101DC00040FF2EC041E050E0082E02C0440F551FD6
:101DD0000A94E2F7942F909592239093F2000EC00C
:101DE000AE9A0895AA9A0895AC9A0895AD9A089566
:101DF000AB9A0895AF9A0895C09A08958430B1F3CC
:101E0000853038F4823081F38330B0F7813041F788
:101E1000E9CF863079F3863058F3873009F7ECCF75
:101E200008950895089508951F920F920FB60F9286
:101E300011242F933F934F935F936F937F938F93CF
:101E40009F93AF93BF93CF93DF93EF93FF93C4B16F
:101E5000D5B1E091F100F0E0EE33F10508F0F7C004
:101E6000E65DFF4FEE0FFF1F0590F491E02D099402
:101E7000D093F500C093F4008091F20080FFE7C09A
:101E8000AE98E5C0D0930B01C0930A018091F20097
:101E900080FFDDC0AE9ADBC085EC87B9D59AD598B6
:101EA000D6C0D093FF00C093FE008091F20085FF62
:101EB000CEC0AA98CCC0D0931501C09314018091D4
:101EC000F20085FFC4C0AA9AC2C080EC87B9D09A3C
:101ED000D098BDC0D093FB00C093FA008091F2006F
:101EE00083FFB5C0AC98B3C0D0931101C09310016B
:101EF0008091F20083FFABC0AC9AA9C086EC87B991
:101F0000D69AD698A4C0D093F700C093F6008091DB
:101F1000F20081FF9CC06BC0D0930D01C0930C01F7
:101F20008091F20081FF93C06CC081EC87B9D19A97
:101F3000D1988DC0D093FD00C093FC008091F20039
:101F400084FF85C0AD9883C0D0931301C093120164
:101F50008091F20084FF7BC0AD9A79C087EC87B98D
:101F6000D79AD79874C0D0930101C0930001809193
:101F7000F20086FF6CC0AB986AC0D0931701C09383
:101F800016018091F20086FF62C0AB9A60C0D093C8
:101F9000F900C093F8008091F20082FF58C0AF981A
:101FA00056C0D0930F01C0930E018091F20082FFC2
:101FB0004EC0AF9A4CC082EC87B9D29AD29847C033
:101FC000D0930301C09302010EC0D0931901C093B6
:101FD000180113C083EC87B9D39AD39838C0D09333
:101FE0000501C09304018091F20087FF30C0C098C2
:101FF0002EC0D0931B01C0931A018091F20087FF7D
:1020000026C0C09A24C084EC21C080910601909122
:10201000070190931D0180931C01D0930701C09389
:1020200006018EE513C00E94030B11C00E945C0BD9
:102030000EC0809108019091090190931F01809337
:102040001E01D0930901C09308018FED87B98091DB
:10205000F1008F5F8093F100833498F01092F100CB
:102060000E94110F8091F3008F5F8093F3008091A5
:10207000200190912101880F991F90932101809355
:10208000200180912001909121018C0F9D1F909340
:10209000210180932001369AFF91EF91DF91CF913A
:1020A000BF91AF919F918F917F916F915F914F9170
:1020B0003F912F910F900FBE0F901F901895809118
:1020C00022018160809322018FEC86B9A69AB89A8A
:1020D000A79AA49AA59AA29AA39A8FE78093F2004E
:1020E0000FB607FE07C08091F3009091F3008917A7
:1020F000E1F314C084EF92E090931D0180931C01E2
:10210000909307018093060189EF90E090931F015F
:1021100080931E0190930901809308010E94D40BC3
:1021200008959C0140E050E060E070E183E190E0C0
:102130000E949415309365002093640008958AE00E
:102140000E943B0EBC0180E094EF0E946D1544E1BB
:1021500050E0649F9001659F300D749F300D1124F5
:10216000C90108950F931F93082F162F81E061E096
:102170000E94A50D82E061E00E94A50D83E061E070
:102180000E94A50D84E061E00E94A50D27E731E0E3
:1021900008C088EE93E0F9013197F1F70197D9F77C
:1021A00001500023B1F781E060E00E94A50D82E0BC
:1021B00060E00E94A50D83E060E00E94A50D84E030
:1021C00060E00E94A50D27E731E008C088EE93E0AB
:1021D000F9013197F1F70197D9F711501123B1F7B0
:1021E0001F910F910895CF93DF9387B38E6187BBC3
:1021F0000E94020C81B38F7081BBF89485E0C7E721
:10220000D1E009C028EE33E0FE013197F1F721500B
:102210003040D1F781508823A9F781E061E00E9426
:10222000B21081E061E00E94B21081E061E00E94A2
:10223000B21082E008C028EE33E0FE013197F1F7DA
:1022400021503040D1F78150B0F783E061E00E9427
:10225000B21083E061E00E94B21083E061E00E946E
:10226000B21082E008C028EE33E0FE013197F1F7AA
:1022700021503040D1F78150B0F781E061E00E94F9
:10228000B21081E061E00E94B21081E063E00E9440
:10229000B2108AE008C028EE33E0FE013197F1F772
:1022A00021503040D1F78150B0F785E0ABCFCF93CC
:1022B000DF93EC018AE00E943B0EC817D90710F4A7
:1022C0000E94F310DF91CF9108958AE00E943B0EA7
:1022D00020916400309165008217930710F00E94EE
:1022E000F3100895089508951F9320912E013091C1
:1022F0002F01620F731F70932F0160932E0123E053
:10230000683E720738F0685E734070932F016093E7
:102310002E018F5F209128013091290140912A01DF
:1023200050912B01280F311D411D511D2093280173
:102330003093290140932A0150932B01909127015A
:10234000980F9093270140E006C0909127019A5082
:102350009093270141E0909127019A30B0F72091A6
:10236000250130912601280F311D3093260120933D
:10237000250110E01EC08091250190912601885E04
:102380009340909326018093250180913001909194
:102390003101A0913201B09133010196A11DB11D0F
:1023A0008093300190933101A0933201B0933301B7
:1023B00011E0809125019091260123E0883E92074B
:1023C000D0F6442311F00E947311112311F00E94E2
:1023D00072111F9108950F931F934FB7F8940091B6
:1023E00028011091290120912A0130912B01800FA1
:1023F000911F009128011091290120912A0130910B
:102400002B019C01201B310B79F020705FEF2030F5
:10241000350751F025B7206425BF78948895F89446
:1024200025B72F7B25BFE5CF4FBF1F910F91089593
:1024300090932401809323012FB7F8948091280171
:1024400090912901A0912A01B0912B012FBF909367
:102450002D0180932C0108953FB7F89480912801B5
:1024600090912901A0912A01B0912B013FBF2091A9
:102470002C0130912D01821B930B2091230130916F
:1024800024018217930718F020E030E002C0281BD7
:10249000390BC90108950E942C120E94EB112FB72D
:1024A000F8948091280190912901A0912A01B0917E
:1024B0002B012FBF90932D0180932C0108958FB78E
:1024C000F894209128013091290140912A015091DE
:1024D0002B018FBFB901CA0108954FB7F8948091BD
:1024E000280190912901A0912A01B0912B019C0112
:1024F0004FBF40918F0050919000241B350B90935B
:10250000900080938F00C9010895CF93DF93CCEFA3
:10251000D1E0CE014FEF5FEF6FEF7FEF0E94ED153F
:102520002497B9F781E0DF91CF9108958F929F9220
:10253000AF92BF92CF92DF92EF92FF920F931F93D1
:10254000CF93DF935B016C01CCEFD1E08CEFE82EF1
:102550008FEFF82E8E01CE010E94C615AB01BC0193
:10256000842F942F91509E3FE8F4242F30E0237065
:1025700030702115310511F08C7F8C5F4A155B0599
:102580006C057D0531F47F6FC8010E94ED1581E077
:102590000AC09701281B3109C20FD31F32E0C03097
:1025A000D307C0F280E0DF91CF911F910F91FF9090
:1025B000EF90DF90CF90BF90AF909F908F90089555
:1025C0004F925F927F928F929F92AF92BF92CF92E3
:1025D000DF92EF92FF920F931F93CF93DF937B01D4
:1025E0008C016A01CCEFD1E09FEF892E912CA12CB8
:1025F000B12C8E209F20A022B1227E2CCE010E94E1
:10260000C615AB01BC01842F4F3F81F4CE01A0E081
:10261000B0E088159905AA05BB0540F1CE01B801C7
:10262000A7010E94F915872DB801A701982F915095
:102630009E3FE0F4282F30E02370307021153105E3
:1026400011F08C7F8C5FC81BD1094E155F056007A8
:10265000710739F45070C601BE010E94CC1581E0AB
:1026600006C0249722E0C030D20740F280E0DF911C
:10267000CF911F910F91FF90EF90DF90CF90BF907F
:10268000AF909F908F907F905F904F900895CF92E2
:10269000DF92EF92FF920F931F93CF93DF937B0113
:1026A0008C016A01CCEFD1E0CE010E94C615AB01CE
:1026B000BC01842F942F91509E3FE0F4242F30E0F2
:1026C000237030702115310511F08C7F8C5FC81B91
:1026D000D1094E155F056007710739F45070C601C6
:1026E000BE010E94B61581E006C0249782E0C0308A
:1026F000D807D0F280E0DF91CF911F910F91FF902A
:10270000EF90DF90CF900895EF92FF920F931F9379
:10271000E82FF0E0A42FB0E0481718F4EA1BFB0BF9
:1027200004C0CD018E1B9F0BFC01872F90E0432F2F
:1027300050E0371728F4DC01A41BB50BAD0102C033
:10274000481B590B862F90E0A22FB0E0261718F4F3
:102750008A1B9B0B04C09D01281B390BC901449F98
:102760009001459F300D549F300D112440E050E002
:10277000EE9F7001EF9FF00CFE9FF00C112400E023
:1027800010E02E0D3F1D401F511F889FB001899FF3
:10279000700D989F700D1124CB01A0E0B0E0280FC0
:1027A000391F4A1F5B1F203080E8380780E0480748
:1027B00080E0580720F02FEF3FE740E050E0C901EC
:1027C0001F910F91FF90EF900895FF920F931F9329
:1027D000CF93DF93F62E532F122F232F30E0C72FE6
:1027E000D0E0751728F4D901AC1BBD0BED0102C078
:1027F000C21BD30B212F30E0EF2DF0E0F11618F4BF
:102800002E1B3F0B04C0DF01A21BB30B9D01922FB7
:10281000021710F000E002C0901B092F841B9927BB
:1028200087FD909597FF03C0909581959F4F90E00D
:10283000889F9001899F300D989F300D1124C90108
:10284000AA2797FDA095BA2F272F30E0250F311D1D
:102850003695279530E040E050E0BC01CD010E9464
:102860004E15272F382F492F5527D0E0CC9FF00148
:10287000CD9FF00DDC9FF00D1124BF01882777FD5F
:102880008095982F620F731F841F951F2F2D30E0A6
:10289000210F311D3695279530E040E050E00E9431
:1028A0004E15672F782F892F992710E0009FF00190
:1028B000019FF00D109FF00D11249F01442737FD5B
:1028C0004095542F260F371F481F591F2030F0E81E
:1028D0003F07F0E04F07F0E05F0720F02FEF3FE702
:1028E00040E050E0C901DF91CF911F910F91FF901F
:1028F00008950F9300E00E94E5130F9108950F9340
:102900001F93CF93DF93382F262FC42FD0E0862F2D
:10291000631708F4832F90E0EC2FC817D9070CF445
:10292000E82F0E2F10E0822F321708F4832F90E04B
:10293000C817D9070CF4CE01081B190BEE2311F4AC
:10294000F0E00FC08FEF90E0BC01069FC001079F31
:10295000900D169F900D11246E2F70E00E946D1542
:10296000F62F0115110509F447C0E317B9F430E05B
:102970002C1B3D0BB801660F771F85E590E0AC017D
:10298000249FC001259F900D349F900D11240E941B
:102990006D1577FF33C060507F4F30C0E217A1F450
:1029A000C31BD109B801660F771F85E590E09C0134
:1029B000C29FC001C39F900DD29F900D11240E9411
:1029C0006D156B5A7F4F1AC0E417B1F4832F90E056
:1029D000821B9109B801660F771F25E530E0AC0135
:1029E000429FC001439F900D529F900D11240E9461
:1029F0006D1565557F4F02C060E070E02F2F30E00D
:102A000040E050E0542F432F322F22278E2F90E0AA
:102A1000A0E0B0E0282B392B4A2B5B2B70E080E044
:102A200090E0CB0177276627262B372B482B592B95
:102A3000B901CA01DF91CF911F910F910895EF92D3
:102A4000FF920F931F93E42E262F30E040E050E0DA
:102A5000542F432F322F2227FF2400E010E02E298D
:102A60003F29402B512B90E0A0E0B0E0DC019927FA
:102A70008827282B392B4A2B5B2BB901CA011F91C0
:102A80000F91FF90EF90089526EA3EE004C0F9010F
:102A90003197F1F701970097D1F70895629FD00120
:102AA000739FF001829FE00DF11D649FE00DF11D09
:102AB000929FF00D839FF00D749FF00D659FF00DB8
:102AC0009927729FB00DE11DF91F639FB00DE11DA5
:102AD000F91FBD01CF0111240895AA1BBB1B51E1B1
:102AE00007C0AA1FBB1FA617B70710F0A61BB70B7E
:102AF000881F991F5A95A9F780959095BC01CD0123
:102B0000089597FB092E07260AD077FD04D0E5DF4C
:102B100006D000201AF4709561957F4F0895F6F75E
:102B2000909581959F4F0895A1E21A2EAA1BBB1B79
:102B3000FD010DC0AA1FBB1FEE1FFF1FA217B30789
:102B4000E407F50720F0A21BB30BE40BF50B661F9F
:102B5000771F881F991F1A9469F760957095809563
:102B600090959B01AC01BD01CF010895DC01CB0123
:102B7000FC01E199FECF06C0FFBBEEBBE09A3196A7
:102B80000DB20D9241505040B8F70895A6E1B0E063
:102B900044E050E00C94B815DC01A40FB51F41507F
:102BA000504048F0CB01840F951F2E910E94DD15F7
:102BB00041505040D0F70895262FE199FECF9FBB9A
:102BC0008EBBE09A01970DB2021631F02DBB0FB605
:102BD000F894E29AE19A0FBE08950396272F0E9477
:102BE000DD150E94DC15252F0E94DD15242F0C9485
:102BF000DD15242F0E940716252F0E9407160C941E
:102C000001160E940616272F0C940716262FE1990D
:102C1000FECF9FBB8EBB2DBB0FB6F894E29AE19A14
:0A2C20000FBE01960895F894FFCF4F
:062C2A001400140051012A
:00000001FF
